:100000000C9471040C948E040C948E040C948E0445
:100010000C948E040C948E040C948E040C948E0418
:100020000C948E040C948E040C947A0E0C948E0412
:100030000C948E040C941D240C948E040C944A246D
:100040000C948E040C948E040C948E040C948E04E8
:100050000C948E0454797065202268656C7022209F
:10006000666F7220636F6D6D616E64206C6973746E
:100070002E0048656174696E67003233300032309B
:10008000300031353000313030003530002C200068
:100090002C20002C20002C20002C200050574D201C
:1000A0003130302025203D200050574D2038302061
:1000B00025203D200050574D2036302025203D2062
:1000C0000050574D2034302025203D200050574D02
:1000D0002032302025203D200020202054203D20AB
:1000E00020004454203D20003530004F7665727367
:1000F000686F6F74203D200000180C0C0C0000AAE3
:10010000050A2A05059A050B040C0A8A05067A05D4
:100110000100000000000000000000000001500D80
:100120006A0A7B0BAA050A8205006105020000012C
:1001300000000000000000000000000000000000BF
:10014000000002F20C670A6D0BAA050A8205006125
:100150000503000002000000000000000000000095
:100160000000000000000003940C640A5F0BAA0565
:100170000A82050061050400000300000000000081
:1001800000000000000000000000000004360C61C8
:100190000A510BAA050A820500610505000004004A
:1001A000000000000000000000000000000000004F
:1001B0000005440B11051205AA050A5605000000AA
:1001C000050000000000000000000000000000002A
:1001D00000000000000006210B5E0A0707AA050ABE
:1001E0009205003505070000060000000000000031
:1001F000000000000000000000000007FE0A5B0A8B
:100200000307AA050A9205002A0508000007000056
:1002100000000000000000000000000000000000DE
:1002200008D30A580AA708AA050A9205004005093A
:1002300000000800000000000000000000000000B6
:10024000000000000009B30A550A6D0AAA050A92C7
:10025000050017050C000009000000000000000068
:10026000000000000000000000000A270CEC0B1644
:1002700005AA050A8A05069A050B040C0A00000067
:100280000000000000000000000000000000000B63
:10029000BC0B520AC208AA050AA205004B050B2096
:1002A000050000000B00000000000000000000003E
:1002B000000000000C890BE3093C08AA050A92051E
:1002C0000000000C00000000000000000000000022
:1002D0000000000000000000002000205472616E49
:1002E00073203A20002000200020537461746520A0
:1002F0003A20006605F406671F6B05F406671F8247
:1003000005EF073B199D050000551DA505000019C7
:100310001DAD050000DC1CB40500009E1CBB0500E3
:1003200000611CC4050000251CCD050000E81BD59C
:10033000050000AA1BDD0500006D1BE8050000316B
:100340001BF3050000F41AFD050000B61A070600AD
:1003500000791A110600003D1A1B060000001A243D
:10036000060000C2198A05D10688192D060D0763FB
:100370001F360657075F1F5A05A707A91E6005CA43
:10038000077F1E71050000281E3F0500001C1E95FA
:10039000050000C51D99050000921D43054C06147B
:1003A0001E480561060C1E53058606F81D4E057392
:1003B00006041E7905A206D31E40061208551E002B
:1003C000000000000032313A30393A3439004D61D2
:1003D00072202034203230303900330031002320A5
:1003E00020436F6D6D616E6473203A200023207589
:1003F0007365202268656C7022002320436F6D6D49
:10040000616E64206E6F7420666F756E64003031AB
:10041000323334353637383941424344454600504B
:100420004342502D5265666C6F7720436F6E747235
:100430006F6C6C657200536F667477617265200033
:1004400056657273696F6E203A200052656C656163
:100450007365203A200044617465203A2000546995
:100460006D65203A200073746172742000726561BA
:100470006479200073656C66746573742000206471
:10048000656743002053656B756E64656E002025BB
:1004900000204B2F68002050686173656E6D6F649B
:1004A000757300204F4E00204F464600204C65617A
:1004B000726E002041646A75737400205072656822
:1004C0006561740020536F616B00204477656C6C2C
:1004D00000205265666C6F77002054656D70657200
:1004E000617475723A00205A6569743A0020416E51
:1004F00073746965673A00204C65697374756E673B
:100500003A00205B30206F64657220315D00205B13
:10051000302E2E3235345D00205B302E2E363535B0
:1005200033345D00205B302E2E3130305D00205B97
:100530002D33323736372E2E33323736365D007054
:10054000656300736F6C64006C6561726E00737438
:100550006F700061646A757374006465627567002A
:1005600074726163650068656C700068696C6665CB
:100570000076657273696F6E0073657474696E6777
:10058000730073686F77616C6C0074656D706F6673
:1005900066736574006E6C670072727300706874C5
:1005A00074656D700070687474696D65007068744E
:1005B00070777200706874696E6300736F616B743A
:1005C000656D7000736F616B74696D6500736F6149
:1005D0006B70777200736F616B696E630072656632
:1005E0006C6F7774656D70007265666C6F77746997
:1005F0006D65007265666C6F777077720072656604
:100600006C6F77696E63006477656C6C74656D7090
:10061000006477656C6C74696D65006477656C6CFB
:10062000707772006477656C6C696E630074656DD9
:100630007073686F770074656D70747261636500C4
:10064000747261646974696F6E616C0020537461C7
:1006500072746574204C6F6574766F7267616E6733
:10066000002053746172746574204C65726E6C6105
:100670007566002053746F7074204C6F6574766FCC
:100680007267616E670020537461727465742053E1
:10069000656E736F726B616C696272696572756E9B
:1006A00067002053656C656B7469657274206465BE
:1006B0006E20616B746976656E20506172616D6544
:1006C0007465727361747A205B20302E2E34205D45
:1006D000002054656D70657261747572204A75737F
:1006E00074616765205B2D33302E2E33305D2047DB
:1006F00072616400204C697374657420616C6C6570
:100700002042656665686C652061756600205465E9
:100710006D7065726174757220696E206A656465BA
:100720007220506861736520616C6C65722058207E
:1007300053656B756E64656E206175736765626580
:100740006E205B506172616D657465722030206F40
:1007500064657220585D002054656D706572617427
:1007600075722077C3A46872656E64206465732017
:100770004CC3B674656E7320616C6C657220582032
:1007800053656B756E64656E206175736765626530
:100790006E205B506172616D657465722030206FF0
:1007A00064657220585D0020446562756767696EF4
:1007B0006720496E666F726D6174696F6E656E2039
:1007C00020617573676562656E0020496E7465729D
:1007D0006E65204175746F6D6174656E7A757374A2
:1007E00061656E646520617573676562656E002082
:1007F000416C6C652045696E7374656C6C756E67D1
:10080000656E20617573676562656E00202D2D3EF3
:100810002000204865697A756E67737265676C653C
:100820007220696D204F6C64205374796C6520765A
:10083000657277656E64656E000D0A4175746F6D43
:100840006174697363686572204C6F657462657466
:1008500072696562206E6F6368206E6963687420D8
:100860006D6F65676C6963682E0D0A426974746503
:100870002065727374204F66656E706172616D657C
:100880007465722065696E6C65726E656E0D0A0026
:100890004269747465206265692000204772616452
:1008A000205461737465204C6561726E20626574BA
:1008B0006165746967656E0041646A75737420626E
:1008C00065656E6465742E204269747465204F6698
:1008D000656E206E65752065696E6C65726E656EFD
:1008E000000011241FBECFE5D8E0DEBFCDBF10E071
:1008F000A0E6B0E0ECE4FEE402C005900D92AA3957
:10090000B107D9F712E0AAE9B0E001C01D92A438FE
:10091000B107E1F70E9490040C9424270C94000086
:100920000E94E20D0E94A9250E9415100E940A0F44
:100930000E94762060E875E280E090E00E94C62484
:100940008BE994E20E942E19789460E875E280E0C9
:1009500090E00E94DB238AEF93E20E94D3228FE192
:1009600094E00E94102386E394E00E94F02280E04D
:1009700090E00E94281E0E94E4160E94BC0D81E0B7
:100980000E94C02280E00E949A2284E794E00E94A4
:10099000F02286E694E00E9410230E948A2582E0DD
:1009A0000E94132588EE93E00E94B0218823D1F79E
:1009B0000E94132584E794E00E94F0228DE694E0E3
:1009C0000E94102384E590E00E94F0220E940323FD
:1009D0000E9449060E94530F80E00E94E10F882385
:1009E00069F00E94B205843021F480E00E94F20593
:1009F00005C00E94C20E82E00E94AD0581E00E9407
:100A0000E10F882319F081E00E94AD0582E00E9489
:100A1000E10F882319F083E00E94AD050E94612058
:100A2000D7CF089581E08093A1000895089520E034
:100A30008091B9009091BA0097FD21E0822F08952E
:100A400020E08091B9009091BA0005970CF421E064
:100A5000822F089520E08091B4009091B500883CE9
:100A600091050CF021E0822F089520E08091B400E0
:100A70009091B500893C91050CF421E0822F0895F6
:100A800020E08091B4009091B500805991400CF025
:100A900021E0822F089520E08091B4009091B5006C
:100AA000815991400CF421E0822F089520E080913B
:100AB000B4009091B500883C91050CF421E0822FA0
:100AC000089560E02091A6003091A7004091A80011
:100AD0005091A9008091AA009091AB00A091AC0028
:100AE000B091AD00281739074A075B0708F061E0AD
:100AF000862F089590E08091A000823009F491E063
:100B0000892F089590E08091A000823009F091E053
:100B1000892F089590E08091A000833009F491E03E
:100B2000892F089590E08091A000833009F091E032
:100B3000892F089590E08091A000843009F491E01D
:100B4000892F089590E08091A000843009F091E011
:100B5000892F089580919B000895853010F480932B
:100B6000A10008958091A00008950F931F93F901AB
:100B700050930E0240930D0260930F027093100287
:100B80008093110290931202509314024093130227
:100B9000CA01880F991F880F991F840F951F62E063
:100BA00070E00E94D4267093160260931502000F25
:100BB000111F000F111F222717FD2095322F0093C0
:100BC0001702109318022093190230931A02EE0FA5
:100BD000FF1FEE0FFF1FF0931C02E0931B021F91FB
:100BE0000F910895982F8091A0008430E9F5992302
:100BF000D9F56091B4007091B50080919A000E947F
:100C0000C31580919A00843021F481E08093A10083
:100C100008958F5F80939A0080E998E00E94F02207
:100C200080919A00823091F0833028F4882341F03B
:100C30008130B1F408C0833061F0843089F40CC095
:100C40008AE890E00BC086E890E008C082E890E077
:100C500005C08EE790E002C08AE790E00E94F02293
:100C60008BE998E00E94102308951F93182F0E948B
:100C70003113882329F08091B800612F0E946C12F3
:100C80001F9108950E9487209093B5008093B4002F
:100C90000895EF92FF920F931F930E94FF0E7B0126
:100CA0008C018091A6009091A700A091A800B0911E
:100CB000A9008E159F05A007B10709F47BC0E0923B
:100CC000A600F092A7000093A8001093A90080E06E
:100CD00090E00E94B02180939B000E9466138823BD
:100CE00009F468C080919C00882319F0815080939A
:100CF0009C0080919C00882309F05CC00E945B13DB
:100D0000882341F08091600090916100875A94405F
:100D100009F450C080916000909161000E94F0221F
:100D200089E990E00E94F0220E94661380939C0063
:100D30008AE066E040E020E20E94152386E990E028
:100D40000E94F022809113029091140264E070E0FE
:100D50000E94D4267B010027F7FC0095102F8AE023
:100D600064E041E020E30E94152383E990E00E94C3
:100D7000F0228EE794E00E94F02280E990E00E9449
:100D8000F0220E94872064E070E00E94D4267B015C
:100D90000027F7FC0095102F8AE064E041E020E393
:100DA0000E9415238DE890E00E94F0228EE794E0E7
:100DB0000E9410238091A2009091A3009093A5001F
:100DC0008093A40062E670E048EB50E00E94A5101A
:100DD0009093A3008093A2002091A4003091A500DD
:100DE0002817390719F080E00E9435069091A1007C
:100DF0008091A000891711F09093A0001F910F918E
:100E0000FF90EF90089580E00E94ED24089580E027
:100E10000E94ED2408956F927F928F929F92AF92DD
:100E2000BF92CF92DF92EF92FF920F931F93CF93D7
:100E3000DF93EC0180E00E945D158C179D0764F143
:100E400080E00E945D155C01CC24B7FCC094DC2CD2
:100E500081E00E945D157C01CE01AA2797FDA09537
:100E6000BA2FA6019501281B390B4A0B5B0BCA014F
:100E7000B9012CEE3FEF4FEF5FEF0E94A126002754
:100E8000F7FC0095102FEA18FB080C091D09A801B2
:100E900097010E94092731C081E00E945D158C17DF
:100EA0009D0784F180E00E945D155C01CC24B7FCB5
:100EB000C094DC2C81E00E945D157C01BE01882776
:100EC00077FD8095982F6A197B098C099D0924E18B
:100ED00030E040E050E00E94A1260027F7FC00959A
:100EE000102FEA18FB080C091D09A80197010E94A0
:100EF0000927C901DA019C01AD012C5E3F4F4F4F1C
:100F00005F4FA4C082E00E945D158C179D0784F19D
:100F100081E00E945D155C01CC24B7FCC094DC2C00
:100F200082E00E945D157C01BE01882777FD8095D7
:100F3000982F6A197B098C099D0924E130E040E073
:100F400050E00E94A1260027F7FC0095102FEA1818
:100F5000FB080C091D09A80197010E940927C90176
:100F6000DA019C01AD01285D3F4F4F4F5F4F6EC0CE
:100F700083E00E945D153E01882477FC8094982CC4
:100F80008C179D076CF182E00E945D155C01CC24FA
:100F9000B7FCC094DC2C83E00E945D157C016A18CC
:100FA0007B088C089D08C401B30124E130E040E0D7
:100FB00050E00E94A1260027F7FC0095102FEA18A8
:100FC000FB080C091D09A80197010E940927C90106
:100FD000DA019C01AD01245C3F4F4F4F5F4F36C09B
:100FE00083E00E945D155C01CC24B7FCC094DC2C2E
:100FF00084E00E945D157C016A187B088C089D08BE
:10100000C401B30124E130E040E050E00E94A12699
:101010000027F7FC0095102FEA18FB080C091D09A2
:10102000A80197010E940927C901DA019C01AD01BD
:10103000205B3F4F4F4F5F4F25363105410551052E
:101040002CF024E630E040E050E006C057FF04C03A
:1010500020E030E040E050E0822FDF91CF911F91FF
:101060000F91FF90EF90DF90CF90BF90AF909F9047
:101070008F907F906F900895EF92FF920F931F9340
:1010800080E00E94ED2480E00E94ED248DEC90E051
:101090000E94F02280E00E945D157C010027F7FC91
:1010A0000095102F8AE065E041E020E20E941523C0
:1010B00081EC90E00E94102381E00E945D157C018C
:1010C0000027F7FC0095102F8AE065E041E020E260
:1010D0000E94152385EB90E00E94102382E00E947D
:1010E0005D157C010027F7FC0095102F8AE065E074
:1010F00041E020E20E94152389EA90E00E9410233B
:1011000083E00E945D157C010027F7FC0095102FFD
:101110008AE065E041E020E20E9415238CE990E03E
:101120000E94102384E00E945D157C010027F7FCDB
:101130000095102F8AE065E041E020E20E9415232F
:101140000E9403231F910F91FF90EF90089580E07C
:101150000E94ED248091B9009091BA009093BC0058
:101160008093BB0024E230E0829FB001839F700D2A
:10117000929F700D112484E00E948E1580E00E94E1
:10118000ED24089580E00E94ED2480E00E94ED248B
:101190008FEF0E944B1588EB98E00E941023089572
:1011A000EF92FF920F931F93CF93DF93C091B40000
:1011B000D091B50080919D0090919E00892B21F4E3
:1011C000D0939E00C0939D000E94E90E90919F00D5
:1011D000882309F4B5C0992309F4B7C080919D0014
:1011E00090919E009E01281B390B89E190E0AC0193
:1011F000249FC001259F900D349F900D1124409194
:10120000B9005091BA009A01220F331F240F351FE5
:10121000820F931F64E070E00E94D4267093BA009E
:101220006093B90010929F000E944613882359F1E1
:1012300082EE90E00E94F022E090B900F090BA00B7
:101240000027F7FC0095102F8AE064E041E020E2DF
:101250000E94152389ED90E00E94F0228091B40055
:101260009091B50064E070E00E94D4267B010027D5
:10127000F7FC0095102F8AE064E041E020E20E9434
:1012800015230E940323D0939E00C0939D00E090FD
:101290001702F09018020091190210911A02609141
:1012A000A6007091A7008091A8009091A9002091BC
:1012B0000F02309110024091110250911202621BF4
:1012C000730B840B950BA80197010E94A12620E1C6
:1012D0003EE040E050E00E94092780910D0290918D
:1012E0000E02820F931F909314028093130217FF34
:1012F00008C020911B0230911C028217930760F4F2
:1013000007C020911B0230911C022817390720F4D6
:10131000309314022093130220911302309114028F
:10132000C901880F991F880F991F820F931F62E0D0
:1013300070E00E94D426709316026093150205C0D7
:10134000992319F481E080939F000E948222182F34
:101350000E94EF14E091B400F091B500811700F500
:1013600040E08091BD0090E02091B9003091BA003A
:10137000BC01629FC001639F900D729F900D11246C
:1013800069E170E00E94D426E60FF71F80911302F6
:1013900090911402E817F9070CF441E0842F0AC079
:1013A00020E08091130290911402E817F9070CF4E1
:1013B00021E0822F0E949022DF91CF911F910F9107
:1013C000FF90EF9008950E94D0088091B400909112
:1013D000B5002091B6003091B700821B930B889620
:1013E00081359105C8F48091A6009091A700A09145
:1013F000A800B091A9002091AE003091AF004091BB
:10140000B0005091B100821B930BA40BB50BCD978C
:10141000A105B10508F445C08091B9009091BA00CA
:1014200024E230E0829FB001839F700D929F700D87
:10143000112480919A000E948E1580919A00833029
:1014400061F48091BD000E944B1588EE93E00E94EC
:10145000832581E08093A10008958F5F80939A0097
:101460000E9482228C5E0E949A228091A600909116
:10147000A700A091A800B091A9008093AE0090931E
:10148000AF00A093B000B093B1008091B4009091F0
:10149000B5009093B7008093B60084E690E00E9478
:1014A000832508950E94D00808950E94D0080895C9
:1014B0000E94D00808950E94D00808950E94D00884
:1014C00008950E94D00808950E94D00808950E94AF
:1014D000D00808950E94D0080895EF92FF920F93CC
:1014E0001F936091B4007091B500882777FD8095B7
:1014F000982F29E130E040E050E00E94A1266051A1
:101500007742804090402091BB003091BC0044273E
:1015100037FD4095542F0E9409272093BD000E945B
:101520004613882389F08BEE90E00E94F022E09031
:10153000BD00FF2400E010E08AE064E041E020E22A
:101540000E9415230E94032380E00E94ED2480E086
:101550000E94132584E690E00E9483251F910F913D
:10156000FF90EF9008950F931F938CEA94E090936F
:1015700061008093600088E00E9413256091A600BE
:101580007091A7008091A8009091A9004091B400AB
:101590005091B5002AE030E000E013E80E94B50564
:1015A0001F910F9108950F931F938CEA94E09093ED
:1015B00061008093600088E00E9413251092BA00B9
:1015C0001092B9001092BC001092BB0084E60E94F9
:1015D0009A226091A6007091A7008091A800909136
:1015E000A9004091B4005091B50022E830E000E03D
:1015F0001DE70E94B5051F910F9108950F931F934A
:101600008CEA94E0909361008093600088E00E94EF
:10161000132584E60E949A226091A6007091A7008B
:101620008091A8009091A9004091B4005091B5001C
:1016300022E830E000E01DE70E94B5051F910F9100
:1016400008950F931F938CEA94E090936100809328
:10165000600080E00E94ED2488E00E9413256091E4
:10166000A6007091A7008091A8009091A9004091D8
:10167000B4005091B5002AE030E000E013E80E9489
:10168000B5051F910F91089587EA94E0909361004A
:101690008093600080E00E949A2283E00E941325DC
:1016A000089580E00E94ED2480E00E94ED2480E017
:1016B0000E94132580EA9FE00E948325089580E020
:1016C0000E94ED2480E00E94ED2480E00E9413251A
:1016D00084E690E00E948325089580E00E94ED2436
:1016E00080E00E94ED2480E00E94132584E690E0D3
:1016F0000E948325089580E00E94ED2480E00E94EE
:10170000132580E00E94ED2488EE93E00E9483255B
:1017100008950F931F938CEA94E090936100809357
:10172000600088E00E9413256091A6007091A700D8
:101730008091A8009091A9006093AE007093AF00D3
:101740008093B0009093B1004091B4005091B500E7
:101750005093B7004093B6002CE231E000E01DE763
:101760000E94B5050E94852284E10E949A2210926F
:101770009A001F910F9108950F931F9383EB94E0AC
:1017800090936100809360000E94F81589E00E94A8
:1017900013256091A6007091A7008091A8009091F8
:1017A000A9004091B4005091B5002CE231E000E076
:1017B0001DE70E94B50510929A0080E998E00E940A
:1017C000F02288EE90E00E94F0228BE998E00E94DF
:1017D00010231F910F91089580919B00882341F061
:1017E0000E941025823079F082E00E94132508952E
:1017F0000E9448158F3F39F40E941025813019F05E
:1018000081E00E94132508950E94481590E08F3FC3
:1018100009F491E0892F08950E9448158F3F39F40B
:101820000E941025813019F081E00E94132508954F
:1018300080E00E94ED2480E00E9413250E9448155C
:101840008093BD008F3F11F41092BD00089587EA88
:1018500094E090936100809360000E948A2280E06F
:101860000E94132581E08093A10008959F92AF927A
:10187000BF92CF92DF92EF92FF920F931F938AEC69
:1018800094E090936100809360000E943C13882351
:1018900019F00E946A1408C00E9496160E940B0755
:1018A000182F0E940415810F0E949A22E090A60032
:1018B000F090A7000091A8001091A9000E94A31623
:1018C000A0E0B0E08E0D9F1DA01FB11F8093AA0065
:1018D0009093AB00A093AC00B093AD00C090A60075
:1018E000D090A700E090A800F090A900A090B400CC
:1018F000B090B5000E945B14982E0E9496168C0141
:10190000C701B601A501292D30E00E94B50587E089
:101910000E9413251F910F91FF90EF90DF90CF90C1
:10192000BF90AF909F9008959F92AF92BF92CF9239
:10193000DF92EF92FF920F931F9381ED94E09093CB
:101940006100809360000E943C13882319F00E947C
:10195000B41408C00E947C160E940B07182F0E9426
:101960000415810F0E949A22E090A600F090A70033
:101970000091A8001091A9000E948916A0E0B0E093
:101980008E0D9F1DA01FB11F8093AA009093AB00E6
:10199000A093AC00B093AD00C090A600D090A7007B
:1019A000E090A800F090A900A090B400B090B5001D
:1019B0000E94A514982E0E947C168C01C701B601C6
:1019C000A501292D30E00E94B50586E00E9413256F
:1019D0001F910F91FF90EF90DF90CF90BF90AF904D
:1019E0009F9008959F92AF92BF92CF92DF92EF9215
:1019F000FF920F931F9384EC94E090936100809387
:101A000060000E943C13882319F00E941B1408C038
:101A10000E94B0160E940B07182F0E940415810F18
:101A20000E949A22E090A600F090A7000091A800E2
:101A30001091A9000E94BD16A0E0B0E08E0D9F1D80
:101A4000A01FB11F8093AA009093AB00A093AC009D
:101A5000B093AD00C090A600D090A700E090A80081
:101A6000F090A900A090B400B090B5000E940714B7
:101A7000982E0E94B0168C01C701B601A501292D30
:101A800030E00E94B50585E00E9413251F910F915B
:101A9000FF90EF90DF90CF90BF90AF909F90089510
:101AA0009F92AF92BF92CF92DF92EF92FF920F93ED
:101AB0001F938BEB94E090936100809360000E94F1
:101AC000C20E1092A6001092A7001092A8001092C9
:101AD000A9000E943C13882319F00E94CA1308C071
:101AE0000E94CA160E940B07182F0E940415810F2E
:101AF0000E949A22E090A600F090A7000091A80012
:101B00001091A9000E94D716A0E0B0E08E0D9F1D95
:101B1000A01FB11F8093AA009093AB00A093AC00CC
:101B2000B093AD00C090A600D090A700E090A800B0
:101B3000F090A900A090B400B090B5000E94B91335
:101B4000982E0E94CA168C01C701B601A501292D45
:101B500030E00E94B50584E00E94132584E690E001
:101B60000E9483251F910F91FF90EF90DF90CF90FF
:101B7000BF90AF909F90089581E08093A0008093E4
:101B8000A10082E690E068EB70E042E750E00E943E
:101B900071119093A3008093A20080E00E9435060B
:101BA0000E941313BC0182E496E00E942F0E9093D2
:101BB000B3008093B2000E9487209093B500809379
:101BC000B4000895EEEBF0E011821082379681E0C8
:101BD000E430F807C9F787E48CBF83B78D6083BF13
:101BE00089B7826089BF0895CF93DF93EC01AEEB94
:101BF000B0E0E0E0F0E08D919C911197892B21F508
:101C00009F0193E0EE0FFF1F9A95E1F7E21BF30BA4
:101C1000E254FF4F168213821282CB0105966AE0CE
:101C200070E00E94C02675836483F894F90183E014
:101C3000EE0FFF1F8A95E1F7E21BF30BE254FF4F13
:101C4000D183C083789407C031961796EA30F105A6
:101C500091F62FEF3FEFC901DF91CF910895CF9318
:101C6000DF93EC01AEEBB0E0E0E0F0E08D919C9111
:101C70001197892B29F59F0153E0EE0FFF1F5A950D
:101C8000E1F7E21BF30BE254FF4F81E086831382FE
:101C90001282CB0105966AE070E00E94C02675832F
:101CA0006483F894F90143E0EE0FFF1F4A95E1F7D2
:101CB000E21BF30BE254FF4FD183C083789407C03B
:101CC00031961796EA30F10589F62FEF3FEFC901FB
:101CD000DF91CF910895F894FC0163E0EE0FFF1FB0
:101CE0006A95E1F7E81BF90BE254FF4F118210826D
:101CF000789408951F920F920FB60F9211242F938C
:101D00003F934F935F936F937F938F939F93AF9383
:101D1000BF93CF93DF93EF93FF93CEEBD0E0888117
:101D20009981892BB9F08A819B8101969B838A8353
:101D30002A813B818C819D812817390758F0E881E1
:101D4000F98109958E81882319F01B821A8202C0BD
:101D500019821882279681E0C430D80701F7FF91D5
:101D6000EF91DF91CF91BF91AF919F918F917F9133
:101D70006F915F914F913F912F910F900FBE0F90F8
:101D80001F901895109208011092090110920A01F3
:101D900010920B01089590E080910401882309F4CA
:101DA00091E090930401992399F08091080190911A
:101DB0000901A0910A01B0910B010196A11DB11D6D
:101DC0008093080190930901A0930A01B0930B013D
:101DD0000895809104010895882371F08091050190
:101DE000882351F41092040181E080930501F89456
:101DF0001DBC1CBC78940895109205010895F894B8
:101E00007894609108017091090180910A01909184
:101E10000B010895109208011092090110920A0115
:101E200010920B018BEC9EE064EF71E00E942F0E8C
:101E300090930701809306011092040181E0809342
:101E40000501F8941DBC1CBC7894089581E0809332
:101E500014010895E82FF0E0EE0FFF1FE45FFE4F3E
:101E60008081662319F0880F816001C0880F80830C
:101E7000808190E08F709070009711F00F9791F42F
:101E80008181662341F080FD02C08560818381816C
:101E90008D7F8183089580FF02C08260818381816C
:101EA0008A7F81830895EF92FF920F931F93809111
:101EB0001401882339F11092140100B3602F60954A
:101EC000661F6627661F80E00E942A0F10E0B80197
:101ED00036E0769567953A95E1F721E0E22EF12C10
:101EE0006E257F25617081E00E942A0F95E016958E
:101EF00007959A95E1F70E251F25017082E0602F66
:101F00000E942A0F1F910F91FF90EF900895E82FE4
:101F1000F0E0EE0FFF1FE45FFE4F818181700895B6
:101F20008091120190911301019690931301809377
:101F30001201039720F010921301109212012091C8
:101F400012013091130140E050E02F5F3F4F2330EA
:101F5000310510F020E030E0922FE22FF0E0EE0F9C
:101F6000FF1FE45FFE4F818180FF06C030931301A5
:101F700020931201892F08954F5F5F4F4330510521
:101F800021F7309313012093120194E0F3CFE82F4F
:101F9000F0E0EE0FFF1FE45FFE4F818190E0969529
:101FA00087959695879581700895E82FF0E0EE0F5C
:101FB000FF1FE45FFE4F818190E0969587958170C9
:101FC0000895E82FF0E0EE0FFF1FE45FFE4F218140
:101FD000822F90E09695879596958795982F91708A
:101FE00080FF02C02B7F2183892F0895E82FF0E026
:101FF000EE0FFF1FE45FFE4F2181822F90E0969548
:102000008795982F917080FF02C02D7F2183892FA3
:102010000895E82FF0E0EE0FFF1FE45FFE4F81818F
:10202000856081838FE08083089581B38F7181BB48
:1020300082B3806E82BB10920C0110920D0110923F
:102040000E0110920F0110921001109211011092C6
:102050001301109212011092140186E29FE06AE0CF
:1020600070E00E942F0E9093160180931501089541
:10207000DF93CF93CDB7DEB72E970FB6F894DEBFC0
:102080000FBECDBF20E030E0AE014F5F5F4FFC01DF
:10209000E20FF31FE491DA01A20FB31FEC932F5F5D
:1020A0003F4F2730310599F7DE011896FA0187E096
:1020B00001900D928150E1F7288539854A855B852D
:1020C0006C857D858E8590E02E960FB6F894DEBFE8
:1020D0000FBECDBFCF91DF910895DF93CF9300D096
:1020E00000D000D0CDB7DEB7FC0184918983319652
:1020F00084918A833196E491EB83DE011496FE018C
:10210000319683E001900D928150E1F76C817D81E1
:102110008E8190E026960FB6F894DEBF0FBECDBF3D
:10212000CF91DF91089580E0089580E0089580E0E8
:10213000089582E00E94E10F089581E00E94E10F7E
:10214000089580E00E94E10F08953F924F925F92C0
:102150006F927F928F929F92AF92BF92CF92DF92B7
:10216000EF92FF920F931F93DF93CF93CDB7DEB71C
:10217000A2970FB6F894DEBF0FBECDBF5C012B0156
:102180003A01FC01028113812081318180E090E0DD
:10219000AE01495F5F4FF901E80FF91FE491DA01E1
:1021A000A80FB91FEC93019687309105A1F7DE01C6
:1021B0001E96FA0187E001900D928150E1F729897E
:1021C0003A893E848B889C88F801849189830F5FCB
:1021D0001F4FF80184918A830F5F1F4FF80184918C
:1021E000025010408B83E980FA80D82E21153105EA
:1021F00011F0F9010995CC24C394E114F10429F0FC
:10220000F7010995882309F43CC0D31409F44FC0A1
:102210008114910411F0F40109950D2D10E0000FC7
:10222000111F000F111F040D151DF80120813181B0
:1022300080E090E0AE014B5E5F4FF901E80FF91FBF
:10224000E491DA01A80FB91FEC930196873091054C
:10225000A1F7DE015C96FA0187E001900D928150B2
:10226000E1F7FC8CED8DFE8D309709F00995611436
:102270007104F1F0F30180816F2D4C2D0E944A1200
:1022800017C00D5F1F4FF80184918C830F5F1F4FA4
:10229000F80184918D830F5F1F4FF80184910250E4
:1022A00010408E83C394EC80FD80D82EA6CF85018C
:1022B000C801A2960FB6F894DEBF0FBECDBFCF9176
:1022C000DF911F910F91FF90EF90DF90CF90BF9023
:1022D000AF909F908F907F906F905F904F903F90C6
:1022E0000895AF92BF92CF92DF92FF920F931F9308
:1022F000DF93CF93CDB7DEB765970FB6F894DEBF07
:102300000FBECDBF8C016B015A01FC0120813181D0
:1023100080E090E0AE01485F5F4FF901E80FF91FE0
:10232000E491DA01A80FB91FEC930196873091056B
:10233000A1F7DE011F96FA0187E001900D9281500E
:10234000E1F7DE011196FE013F9687E001900D92C4
:102350008150E1F7EA81FB81F980309709F0099516
:10236000C114D10431F08F2DB5010E94EE11F60198
:102370008083C80165960FB6F894DEBF0FBECDBF4F
:10238000CF91DF911F910F91FF90DF90CF90BF9081
:10239000AF900895109218011092170110922C011D
:1023A00010922B011092400110923F0110925401A3
:1023B0001092530110926801109267010895E7E1AD
:1023C000F1E020E080819181892B09F02F5F7496E4
:1023D00081E0EB37F807B1F7822F0895482F611598
:1023E000710509F43FC0E7E1F1E020E030E08081D1
:1023F0009181892B89F584E190E0289FD001299F64
:10240000B00D389FB00D1124A95EBE4F11967C937C
:102410006E93F901EE0FFF1FC90163E0880F991F4A
:102420006A95E1F7E80FF91FEE0FFF1FE75EFE4F19
:1024300081E08083FD011382F901EE0FFF1FEE0F93
:10244000FF1FE20FF31FEE0FFF1FEE0FFF1FE55EF2
:10245000FE4F4083822F08952F5F3F4F74962530A3
:10246000310529F68FEF08958F3F99F085308CF470
:10247000282F332727FD309584E190E0289FF00135
:10248000299FF00D389FF00D1124E95EFE4F118257
:1024900010820895E82F8F3FF1F08530E4F484E155
:1024A000E802D0011124A95EBE4FFD018381E80F2F
:1024B000F11D44878F5FFD018383883009F4138207
:1024C000FD018281883010F48F5F8283FD0183815A
:1024D000E80FF11D64830895CF92DF92EF92FF928F
:1024E0000F931F93CF93DF93482F8F3F09F47EC044
:1024F00085300CF07BC0282F332727FD309584E1F1
:1025000090E0289FF001299FF00D389FF00D1124D5
:10251000E95EFE4F80819181892B09F467C084E1D7
:102520004802E0011124C95EDE4F888199810E9432
:10253000F02289EE92E00E94F0228A81883010F425
:10254000DD2402C0DB80D394CC2417C088E0D816E9
:1025500009F4DD24FE01ED0DF11DE480FF2400E00F
:1025600010E0D3948AE062E040E020E30E9415236B
:1025700087EE92E00E94F022C3948A81C81630F35D
:1025800085EE92E00E94F0228A81882369F18830EA
:1025900010F4DD2402C0DB80D3940E9403238881E1
:1025A00099810E94F0228BED92E00E94F022CC24CF
:1025B000C39417C088E0D81609F4DD24FE01ED0DA0
:1025C000F11DE484FF2400E010E0D3948AE062E08F
:1025D00040E020E30E94152389ED92E00E94F02262
:1025E000C3948A81C81630F30E940323DF91CF91F0
:1025F0001F910F91FF90EF90DF90CF9008959C0175
:10260000E199FECF3FBB2EBBE09A8DB308959C01AC
:10261000E199FECF3FBB2EBB6DBB0FB6F894E29A9B
:10262000E19A0FBE089588EC90E0089590917D01A5
:10263000662311F0982B02C08095982390937D011A
:1026400020917D01E199FECFE199FECF84E990E0F0
:102650009FBB8EBB2DBB0FB6F894E29AE19A0FBEDA
:10266000089580917D018695869581700895682FE3
:1026700084E00E941613089580917D0186958170F3
:102680000895682F82E00E941613089580917D01BD
:1026900086958695869581700895682F88E00E94BA
:1026A0001613089580917D0181700895682F81E04F
:1026B0000E941613089580917D0182958F7081701C
:1026C0000895682F80E10E9416130895E199FECFC6
:1026D00083E990E09FBB8EBBE09A8DB30895282FCD
:1026E000E199FECFE199FECF83E990E09FBB8EBBDD
:1026F0002DBB0FB6F894E29AE19A0FBE0895E199C6
:10270000FECF8FE890E09FBB8EBBE09A8DB308951B
:10271000282F853080F480937B01E199FECFE199E9
:10272000FECF8FE890E09FBB8EBB2DBB0FB6F89419
:10273000E29AE19A0FBE0895E199FECF80E990E018
:102740009FBB8EBBE09A8DB30895282F853080F40F
:1027500080937C01E199FECFE199FECF80E990E082
:102760009FBB8EBB2DBB0FB6F894E29AE19A0FBEC9
:10277000089590917B01E199FECF8CE0989FC00174
:102780001124880F991F875E9F4F9FBB8EBBE09AD5
:102790008DB3089590917B01E199FECF88E1989FD8
:1027A000C0011124845E9F4F9FBB8EBBE09A8DB306
:1027B0000895282F90917B01E199FECFE199FECFFA
:1027C0008CE0989FC0011124880F991F875E9F4F4E
:1027D0009FBB8EBB2DBB0FB6F894E29AE19A0FBE59
:1027E0000895282F90917B01E199FECFE199FECFCA
:1027F00088E1989FC0011124845E9F4F9FBB8EBBD0
:102800002DBB0FB6F894E29AE19A0FBE089590910D
:102810007B01E199FECF83E0989FC001112443E042
:10282000880F991F4A95E1F7815E9F4F9FBB8EBB32
:10283000E09A8DB3089590917B01E199FECF88E1F4
:10284000989FC00111248E5D9F4F9FBB8EBBE09A65
:102850008DB30895282F90917B01E199FECFE199E6
:10286000FECF83E0989FC001112453E0880F991F89
:102870005A95E1F7815E9F4F9FBB8EBB2DBB0FB674
:10288000F894E29AE19A0FBE0895282F90917B0167
:10289000E199FECFE199FECF88E1989FC001112414
:1028A0008E5D9F4F9FBB8EBB2DBB0FB6F894E29AF7
:1028B000E19A0FBE089590917B01E199FECF88E1E6
:1028C000989FC0011124855D9F4F9FBB8EBBE09AEE
:1028D0008DB3089590917B01E199FECF88E1989F97
:1028E000C0011124825D9F4F9FBB8EBBE09A8DB3C8
:1028F0000895282F90917B01E199FECFE199FECFB9
:1029000088E1989FC0011124855D9F4F9FBB8EBBBE
:102910002DBB0FB6F894E29AE19A0FBE0895282FC6
:1029200090917B01E199FECFE199FECF88E1989FDC
:10293000C0011124825D9F4F9FBB8EBB2DBB0FB684
:10294000F894E29AE19A0FBE089590917B01E19983
:10295000FECF88E1989FC00111248B5D9F4F9FBBE4
:102960008EBBE09A8DB3089590917B01E199FECFE3
:1029700088E1989FC0011124885D9F4F9FBB8EBB4B
:10298000E09A8DB30895282F90917B01E199FECFB5
:10299000E199FECF88E1989FC00111248B5D9F4F84
:1029A0009FBB8EBB2DBB0FB6F894E29AE19A0FBE87
:1029B0000895282F90917B01E199FECFE199FECFF8
:1029C00088E1989FC0011124885D9F4F9FBB8EBBFB
:1029D0002DBB0FB6F894E29AE19A0FBE089580914C
:1029E0007E010895282F80937E01E199FECFE19921
:1029F000FECF85E990E09FBB8EBB2DBB0FB6F89450
:102A0000E29AE19A0FBE089580917F010895282FE0
:102A100080937F01E199FECFE199FECF86E990E0B6
:102A20009FBB8EBB2DBB0FB6F894E29AE19A0FBE06
:102A30000895809180019091810108958230C1F0C4
:102A4000833028F4882351F0813029F40CC083307E
:102A5000A1F08430B9F020E030E018C0209182016C
:102A60003091830113C020918401309185010EC003
:102A7000209186013091870109C020918801309111
:102A8000890104C020918A0130918B01C901089508
:102A900080918C010895282F80938C01E199FECFBD
:102AA000E199FECF8CE090E09FBB8EBB2DBB0FB6B3
:102AB000F894E29AE19A0FBE08958230C1F0833013
:102AC00028F4882351F0813029F40CC08330A1F020
:102AD0008430B9F020E030E018C020918D013091B1
:102AE0008E0113C020918F01309190010EC0209172
:102AF00091013091920109C020919301309194018C
:102B000004C02091950130919601C9010895E19981
:102B1000FECF47E053E10E94842608958230D1F031
:102B2000833028F4882341F0813061F50CC0833074
:102B3000C1F0843039F51EC070938E0160938D0111
:102B40008DE090E014C07093900160938F018FE04E
:102B500090E00DC0709392016093910181E190E04B
:102B600006C0709394016093930183E190E00E940A
:102B700087150895709396016093950185E190E023
:102B80000E94871508958230D1F0833028F488237D
:102B900041F0813061F50CC08330C1F0843039F5EB
:102BA0001EC0709383016093820182E090E014C0A4
:102BB000709385016093840184E090E00DC0709370
:102BC00087016093860186E090E006C070938901DA
:102BD0006093880188E090E00E94871508957093C3
:102BE0008B0160938A018AE090E00E948715089526
:102BF00080E068EC70E00E94C31581E060E971E05C
:102C00000E94C31582E068E572E00E94C31583E06C
:102C100060E273E00E94C31584E068E973E00E94FB
:102C2000C3150895BC01909381018093800180E0D9
:102C300090E00E9487150895BC0180917B0128E1F6
:102C4000829FC00111248A5D9F4F0E9487150895BD
:102C5000BC0180917B0128E1829FC00111248D5D20
:102C60009F4F0E9487150895BC0180917B0128E148
:102C7000829FC0011124845D9F4F0E948715089593
:102C8000BC0180917B0128E1829FC0011124875DF6
:102C90009F4F0E9487150895BC0180917B0128E118
:102CA000829FC0011124805E9F4F0E948715089566
:102CB000BC0180917B0128E1829FC0011124835EC9
:102CC0009F4F0E9487150895BC0180917B0128E1E8
:102CD000829FC0011124865E9F4F0E948715089530
:102CE000BC0180917B0128E1829FC0011124895E93
:102CF0009F4F0E948715089580917B0128E1829F54
:102D0000C00111248A5D9F4F6FEF72E10E946E2611
:102D1000089580917B0128E1829FC00111248D5D7F
:102D20009F4F6FEF72E10E946E26089580917B01A4
:102D300028E1829FC0011124845D9F4F6FEF72E1F3
:102D40000E946E26089580917B0128E1829FC00138
:102D50001124875D9F4F6FEF72E10E946E260895E8
:102D600080917B0128E1829FC0011124805E9F4FEA
:102D70006FEF72E10E946E26089580917B0128E139
:102D8000829FC0011124835E9F4F6FEF72E10E940A
:102D90006E26089580917B0128E1829FC001112455
:102DA000865E9F4F6FEF72E10E946E2608958091BC
:102DB0007B0128E1829FC0011124895E9F4F6FEF44
:102DC00072E10E946E260895CF92DF92EF92FF92F9
:102DD0000F931F93CF93DF93E199FECFE199FECF3D
:102DE00021E930E03FBB2EBBE09A8DB38F3F09F065
:102DF0008CC1E199FECFE199FECF8FE890E09FBBB7
:102E00008EBB1DBA0FB6F894E29AE19A0FBEE19913
:102E1000FECFE199FECF3FBB2EBB81E08DBB0FB64D
:102E2000F894E29AE19A0FBEE199FECFE199FECFC4
:102E300082E990E09FBB8EBB1DBA0FB6F894E29A70
:102E4000E19A0FBEE199FECFE199FECF83E990E0D0
:102E50009FBB8EBB1DBA0FB6F894E29AE19A0FBEE3
:102E6000E199FECFE199FECF84E990E09FBB8EBB54
:102E70001DBA0FB6F894E29AE19A0FBEE199FECF1F
:102E8000E199FECF85E990E09FBB8EBB85E58DBBC8
:102E90000FB6F894E29AE19A0FBEE199FECFE1995C
:102EA000FECF86E990E09FBB8EBB8AE08DBB0FB65C
:102EB000F894E29AE19A0FBEE199FECFE199FECF34
:102EC0008CE090E09FBB8EBB8FEF8DBB0FB6F8946C
:102ED000E29AE19A0FBE80E090E060EF7FEF0E94FF
:102EE00087150E94F815C0E0D0E0FDE7CF2EE5E59C
:102EF000DE2E7FEAE72E10E508EE64E6F62ECE0120
:102F0000880F991F8C0F9D1F43E0880F991F4A95CA
:102F1000E1F7895E9F4F66E970E00E948715E199AD
:102F2000FECFE199FECFCE01880F991F8C0F9D1F18
:102F300023E0880F991F2A95E1F79C01275E3F4FF8
:102F40003FBB2EBBCDBA0FB6F894E29AE19A0FBE02
:102F5000865E9F4F60E17EE00E948715E199FECF7B
:102F6000E199FECFCE01880F991F8C0F9D1FF3E0D2
:102F7000880F991FFA95E1F79C01245E3F4F3FBBF4
:102F80002EBBDDBA0FB6F894E29AE19A0FBE835ECB
:102F90009F4F6AE570E00E948715E199FECFE199A5
:102FA000FECFCE01880F991F8C0F9D1F73E0880FF5
:102FB000991F7A95E1F79C01215E3F4F3FBB2EBBE5
:102FC000EDBA0FB6F894E29AE19A0FBE805E9F4F79
:102FD00060E17EE00E948715E199FECFE199FECF86
:102FE000CE01880F991F8C0F9D1F43E0880F991FFA
:102FF0004A95E1F79C012E5D3F4F3FBB2EBB1DBBA9
:103000000FB6F894E29AE19A0FBE8D5D9F4F6CE87F
:1030100070E00E948715E199FECFE199FECFCE01C5
:10302000880F991F8C0F9D1F23E0880F991F2A95E9
:10303000E1F79C012B5D3F4F3FBB2EBB0DBB0FB695
:10304000F894E29AE19A0FBE8A5D9F4F60E27CE1BC
:103050000E948715E199FECFE199FECFCE01880F3E
:10306000991F8C0F9D1FA3E0880F991FAA95E1F768
:103070009C01285D3F4F3FBB2EBBFDBA0FB6F894B5
:10308000E29AE19A0FBE875D9F4F68E270E00E946E
:103090008715E199FECFE199FECFCE01880F991FE8
:1030A0008C0F9D1FE3E0880F991FEA95E1F79C01C3
:1030B000255D3F4F3FBB2EBB0DBB0FB6F894E29A88
:1030C000E19A0FBE845D9F4F68E671E00E9487150C
:1030D000E199FECFE199FECFCE01880F991F8C0FA9
:1030E0009D1F63E0880F991F6A95E1F7825D9F4FEE
:1030F0009FBB8EBB1DBB0FB6F894E29AE19A0FBE40
:103100002196C530D10509F0FACEE199FECF8FE8BE
:1031100090E09FBB8EBBE09A8DB380937B01E199D9
:10312000FECF84E990E09FBB8EBBE09A8DB3809385
:103130007D01E199FECF85E990E09FBB8EBBE09ACF
:103140008DB380937E01E199FECF86E990E09FBB2D
:103150008EBBE09A8DB380937F0180E090E06FEFAB
:1031600072E10E946E26909381018093800182E03B
:1031700090E06FEF72E10E946E269093830180933E
:10318000820184E090E06FEF72E10E946E269093DE
:1031900085018093840186E090E06FEF72E10E94E8
:1031A0006E26909387018093860188E090E06FEF10
:1031B00072E10E946E2690938901809388018AE0D3
:1031C00090E06FEF72E10E946E2690938B018093E6
:1031D0008A01E199FECF0CE010E01FBB0EBBE09A24
:1031E0008DB380938C01C80101966FEF72E10E944C
:1031F0006E2690938E0180938D01C80103966FEF28
:1032000072E10E946E269093900180938F01C80115
:1032100005966FEF72E10E946E2690939201809363
:103220009101C80107966FEF72E10E946E2690939C
:10323000940180939301C80109966FEF72E10E9497
:103240006E269093960180939501DF91CF911F9107
:103250000F91FF90EF90DF90CF9008959093A6018B
:103260008093A5018DE192E090936F0280936E02AE
:1032700010921D020895CF92DF92EF92FF920F936A
:103280001F93DF93CF93CDB7DEB727970FB6F89490
:10329000DEBF0FBECDBF19828E010E5F1F4FC8016A
:1032A00063EF72E046E050E00E945026FF246E017A
:1032B0000894C11CD11CE02E012F16E016C0EE812F
:1032C000FF81309731F08C819D81892B11F4C601EB
:1032D0000995F394F19EB00111246D507D4F8E2D10
:1032E000902F46E050E00E9450268A819B81892BD6
:1032F00031F727960FB6F894DEBF0FBECDBFCF9142
:10330000DF911F910F91FF90EF90DF90CF90089584
:10331000EF92FF920F931F93CF93DF93EC018AE814
:1033200095E00E94F0222097F1F08881882349F0EF
:10333000CE010E943226880F991F880F991F0E9484
:1033400012160E94191564E070E00E94D4267B01D9
:103350000027F7FC0095102F8AE065E041E020E2AD
:103360000E94152304C08CE098E00E94F02281EDB9
:1033700096E00E941023DF91CF911F910F91FF9053
:10338000EF900895EF92FF920F931F93CF93DF93E7
:10339000EC0184E296E00E94F0222097B1F088814F
:1033A000882329F0CE010E9432260E9434160E9402
:1033B00096167C010027F7FC0095102F8AE066E046
:1033C00041E020E20E94152304C08CE098E00E94B6
:1033D000F0228AEC94E00E94F0228DEE94E00E94AC
:1033E000F0228EE295E00E94F02281E994E00E94B2
:1033F0001023DF91CF911F910F91FF90EF900895CF
:10340000EF92FF920F931F93CF93DF93EC018BE129
:1034100096E00E94F0222097A9F08881882329F065
:10342000CE010E9432260E948F140E946A14E82E58
:10343000FF2400E010E08AE065E040E020E20E9426
:10344000152304C08CE098E00E94F0228AEC94E0FE
:103450000E94F02287EF94E00E94F0228EE095E037
:103460000E94F0228EE894E00E941023DF91CF9119
:103470001F910F91FF90EF900895EF92FF920F939D
:103480001F93CF93DF93EC0181E196E00E94F0223D
:103490002097A1F08881882329F0CE010E9432264E
:1034A0000E9440160E94A3167C0100E010E08AE012
:1034B0006AE040E020E20E94152304C08CE098E01E
:1034C0000E94F0228AEC94E00E94F02286EE94E0C2
:1034D0000E94F02288E195E00E94F02284E894E0C6
:1034E0000E941023DF91CF911F910F91FF90EF90D9
:1034F0000895EF92FF920F931F93CF93DF93EC0108
:1035000087E096E00E94F0222097A9F08881882326
:1035100029F0CE010E9432260E9479140E945B1489
:10352000E82EFF2400E010E08AE065E040E020E2C1
:103530000E94152304C08CE098E00E94F0228AECDF
:1035400094E00E94F02289ED94E00E94F0228EE047
:1035500095E00E94F0228EE794E00E941023DF9114
:10356000CF911F910F91FF90EF900895EF92FF92EE
:103570000F931F93CF93DF93EC018DEF95E00E94A3
:10358000F0222097B1F08881882329F0CE010E9493
:1035900032260E941C160E947C167C010027F7FC34
:1035A0000095102F8AE066E041E020E20E9415239A
:1035B00004C08CE098E00E94F02281ED94E00E942B
:1035C000F0228DEE94E00E94F0228EE295E00E94BF
:1035D000F02281E994E00E941023DF91CF911F91A6
:1035E0000F91FF90EF900895EF92FF920F931F932A
:1035F000CF93DF93EC0183EF95E00E94F0222097B8
:10360000A9F08881882329F0CE010E9432260E94E9
:10361000D9140E94B414E82EFF2400E010E08AE0E0
:1036200065E040E020E20E94152304C08CE098E0B1
:103630000E94F02281ED94E00E94F02287EF94E056
:103640000E94F0228EE095E00E94F0228EE894E045
:103650000E941023DF91CF911F910F91FF90EF9067
:103660000895EF92FF920F931F93CF93DF93EC0196
:1036700088EE95E00E94F0222097A1F088818823AF
:1036800029F0CE010E9432260E9428160E94891637
:103690007C0100E010E08AE06AE040E020E20E9465
:1036A000152304C08CE098E00E94F02281ED94E0A4
:1036B0000E94F02286EE94E00E94F02288E195E0DC
:1036C0000E94F02284E894E00E941023DF91CF91C1
:1036D0001F910F91FF90EF900895EF92FF920F933B
:1036E0001F93CF93DF93EC018DED95E00E94F022C4
:1036F0002097A9F08881882329F0CE010E943226E4
:103700000E94C3140E94A514E82EFF2400E010E0DC
:103710008AE065E040E020E20E94152304C08CE0CE
:1037200098E00E94F02281ED94E00E94F02289ED61
:1037300094E00E94F0228EE095E00E94F0228EE755
:1037400094E00E941023DF91CF911F910F91FF9081
:10375000EF900895EF92FF920F931F93CF93DF9313
:10376000EC0185ED95E00E94F0222097B1F0888170
:10377000882329F0CE010E9432260E944C160E9416
:10378000B0167C010027F7FC0095102F8AE066E058
:1037900041E020E20E94152304C08CE098E00E94E2
:1037A000F02284EC94E00E94F0228DEE94E00E94DE
:1037B000F0228EE295E00E94F02281E994E00E94DE
:1037C0001023DF91CF911F910F91FF90EF900895FB
:1037D000EF92FF920F931F93CF93DF93EC018DEC49
:1037E00095E00E94F0222097A9F08881882329F093
:1037F000CE010E9432260E9445140E941B14E82E1E
:10380000FF2400E010E08AE065E040E020E20E9452
:10381000152304C08CE098E00E94F02284EC94E030
:103820000E94F02287EF94E00E94F0228EE095E063
:103830000E94F0228EE894E00E941023DF91CF9145
:103840001F910F91FF90EF900895EF92FF920F93C9
:103850001F93CF93DF93EC0184EC95E00E94F0225C
:103860002097A1F08881882329F0CE010E9432267A
:103870000E9458160E94BD167C0100E010E08AE00C
:103880006AE040E020E20E94152304C08CE098E04A
:103890000E94F02284EC94E00E94F02286EE94E0F4
:1038A0000E94F02288E195E00E94F02284E894E0F2
:1038B0000E941023DF91CF911F910F91FF90EF9005
:1038C0000895EF92FF920F931F93CF93DF93EC0134
:1038D0008BEB95E00E94F0222097A9F08881882345
:1038E00029F0CE010E9432260E942A140E94071459
:1038F000E82EFF2400E010E08AE065E040E020E2EE
:103900000E94152304C08CE098E00E94F02284EC11
:1039100094E00E94F02289ED94E00E94F0228EE073
:1039200095E00E94F0228EE794E00E941023DF9140
:10393000CF911F910F91FF90EF900895EF92FF921A
:103940000F931F93CF93DF93EC0184EB95E00E94DC
:10395000F0222097B1F08881882329F0CE010E94BF
:1039600032260E9464160E94CA167C010027F7FCCA
:103970000095102F8AE066E041E020E20E941523C6
:1039800004C08CE098E00E94F0228BEB94E00E944F
:10399000F0228DEE94E00E94F0228EE295E00E94EB
:1039A000F02281E994E00E941023DF91CF911F91D2
:1039B0000F91FF90EF900895EF92FF920F931F9356
:1039C000CF93DF93EC018DEA95E00E94F0222097DF
:1039D000A9F08881882329F0CE010E9432260E9416
:1039E000F1130E94CA13E82EFF2400E010E08AE0E1
:1039F00065E040E020E20E94152304C08CE098E0DE
:103A00000E94F0228BEB94E00E94F02287EF94E07A
:103A10000E94F0228EE095E00E94F0228EE894E071
:103A20000E941023DF91CF911F910F91FF90EF9093
:103A30000895EF92FF920F931F93CF93DF93EC01C2
:103A400085EA95E00E94F0222097A1F088818823E2
:103A500029F0CE010E9432260E9470160E94D716CD
:103A60007C0100E010E08AE06AE040E020E20E9491
:103A7000152304C08CE098E00E94F0228BEB94E0C8
:103A80000E94F02286EE94E00E94F02288E195E008
:103A90000E94F02284E894E00E941023DF91CF91ED
:103AA0001F910F91FF90EF900895EF92FF920F9367
:103AB0001F93CF93DF93EC018DE995E00E94F022F4
:103AC0002097A9F08881882329F0CE010E94322610
:103AD0000E94D9130E94B913E82EFF2400E010E0E1
:103AE0008AE065E040E020E20E94152304C08CE0FB
:103AF00098E00E94F0228BEB94E00E94F02289ED86
:103B000094E00E94F0228EE095E00E94F0228EE781
:103B100094E00E941023DF91CF911F910F91FF90AD
:103B2000EF900895EF92FF920F931F93CF93DF933F
:103B3000EC01009719F189E995E00E94F022888153
:103B4000882341F0CE010E943226853608F084E6B3
:103B50000E9407150E940415E82EFF2400E010E0E3
:103B60008AE064E040E020E20E9415238CE098E0C7
:103B70000E94F0228EE894E00E941023DF91CF9102
:103B80001F910F91FF90EF900895EF92FF920F9386
:103B90001F93CF93DF93EC01009719F185E995E02E
:103BA0000E94F0228881882341F0CE010E943226B3
:103BB000853608F084E60E94F2140E94EF14E82E85
:103BC000FF2400E010E08AE064E040E020E20E9490
:103BD00015238CE098E00E94F0228EE894E00E9489
:103BE0001023DF91CF911F910F91FF90EF900895D7
:103BF00083E595E00E9410230E94B205813019F4FC
:103C000084E00E94AD0508958EE495E00E941023A3
:103C100081E00E940910089588E495E00E94102335
:103C200082E00E940910089583E495E00E94102329
:103C300080E00E9409100895FC01009741F090E097
:103C40008081813309F491E0892F0E9456130895F1
:103C500080E494E00E94F0228CED93E00E94F02238
:103C60000E9403238BE494E00E94F0228AED93E00B
:103C70000E94F0220E94032386E594E00E94F02235
:103C80008EEC93E00E94F0220E94032386E394E0EE
:103C90000E94F0228EE594E00E94F02285EC93E0F1
:103CA0000E94F0220E9403230895CF93DF93EC013A
:103CB00080E496E00E94F022209791F0888188238A
:103CC00029F0CE010E9432260E9441130E943C132B
:103CD000882319F083EA94E005C087EA94E002C0E3
:103CE0008CE098E00E94F02282E198E00E94F022AD
:103CF00082E095E00E941023DF91CF910895CF9349
:103D0000DF93EC0180E695E00E94F022209791F08D
:103D10008881882329F0CE010E9432260E94371321
:103D20000E943113882319F083EA94E005C087EAE2
:103D300094E002C08CE098E00E94F0228AEC97E0C8
:103D40000E94F02282E095E00E941023DF91CF9143
:103D50000895CF93DF93EC018AE595E00E94F0226D
:103D6000209791F08881882329F0CE010E94322685
:103D70000E944D130E944613882319F083EA94E0B1
:103D800005C087EA94E002C08CE098E00E94F0222F
:103D900087EA97E00E94F02282E095E00E941023DB
:103DA000DF91CF910895EF92FF920F931F93CF93DE
:103DB000DF93EC0189E795E00E94F0222097A9F0BB
:103DC0008881882329F0CE010E9432260E94881320
:103DD0000E947F13E82EFF2400E010E08AE064E0F8
:103DE00040E020E20E94152304C08CE098E00E948D
:103DF000F02282EA96E00E941023DF91CF911F917A
:103E00000F91FF90EF900895EF92FF920F931F9301
:103E1000CF93DF93EC01162F88818823A1F1CE0187
:103E20000E9432260E946F13812F0E9461138DE23F
:103E300096E00E94F022CE010E943226892B29F4BE
:103E400087EA94E00E94102310C00E946613E82EB7
:103E5000FF2400E010E08AE064E040E020E20E94FD
:103E6000152384E894E00E94F02286E994E00E9401
:103E7000F0220E945B13882319F083EA94E016C0B5
:103E800087EA94E013C00E94872064E070E00E94FB
:103E9000D4267B010027F7FC0095102F8AE064E010
:103EA00041E020E20E9415238EE794E00E94102357
:103EB000DF91CF911F910F91FF90EF90089561E0F6
:103EC0000E94041F089560E00E94041F08951F933C
:103ED0008EED93E00E94102310929D0187E991E0FE
:103EE00063EF72E046E050E00E94502616E02BC0DF
:103EF0008091990190919A01892B71F0C9010E94DA
:103F0000F0228CE098E00E94F0228091990190913B
:103F10009A010E94102307C0E0919B01F0919C013F
:103F200080E090E0099560919D016F5F60939D0135
:103F3000619FB00111246D507D4F87E991E046E00B
:103F400050E00E9450262091970130919801211550
:103F5000310571F60E9448158F3F21F489E398E0FE
:103F60000E94F0221F910895DF92EF92FF920F932B
:103F70001F93DF93CF93CDB7DEB764970FB6F89456
:103F8000DEBF0FBECDBF1092A4018EE991E063EFBA
:103F900072E046E050E00E9450267E010894E11C49
:103FA000F11C36E0D32E2FC0C7010E945926F7011D
:103FB00001900020E9F78F01015010400E191F09F0
:103FC000C7016DE172E0A8010E946026009759F4D4
:103FD000E091A201F091A301309721F1C801835E25
:103FE0009D4F09951FC06091A4016F5F6093A4016C
:103FF0006D9DB00111246D507D4F8EE991E046E03A
:1040000050E00E94502660919E0170919F016115C1
:10401000710551F68AEF93E00E9410238DEE93E034
:104020000E94102364960FB6F894DEBF0FBECDBF7A
:10403000CF91DF911F910F91FF90EF90DF90089546
:104040001F93182F0E94D8221A30A1F01D3091F032
:10405000E0916E02F0916F02183009F522E0ED3127
:10406000F20769F160F13197F0936F02E0936E020D
:10407000108225C080916E0290916F028D51924006
:10408000F1F0E8F00E9403230E94B41F8DE192E05A
:1040900090936F0280936E0210921D0210C082E016
:1040A000ED36F80760F41083E0916E02F0916F0234
:1040B0003196F0936F02E0936E02319711821F9157
:1040C0000895DF93CF930F92CDB7DEB7E091A501AE
:1040D000F091A601CE0101960995882319F08981F6
:1040E0000E9420200F90CF91DF910895A19884B372
:1040F000816484BBA898AE9AA99808958091A8017C
:104100008F5F8093A80108958091A70108956F9211
:104110007F928F929F92AF92BF92CF92DF92EF9257
:10412000FF920F931F93CF93DF93A898AE98C0E0B0
:10413000D0E080E0A89ACC0FDD1F99992196A8982D
:104140008F5F8D30B9F7A89A0E941915C80FD91F33
:1041500080E00E941E158C179D0740F180E00E94B0
:104160001E155C01CC24DD2481E00E941E157C011B
:10417000CE01AA2797FDA095BA2FA6019501281B6D
:10418000390B4A0B5B0BCA01B90128E33FEF4FEF34
:104190005FEF0E94A12600E010E0EA18FB080C097E
:1041A0001D09A80197010E9409272DC081E00E94E6
:1041B0001E158C179D0760F180E00E941E155C01A2
:1041C000CC24DD2481E00E941E157C01BE018827DD
:1041D00077FD8095982F6A197B098C099D0928EC39
:1041E00030E040E050E00E94A12600E010E0EA1834
:1041F000FB080C091D09A80197010E940927C901A4
:10420000DA019C01AD0128533F4F4F4F5F4F8EC0E5
:1042100082E00E941E158C179D0760F181E00E94CC
:104220001E155C01CC24DD2482E00E941E157C0159
:10423000BE01882777FD8095982F6A197B098C0924
:104240009D0928EC30E040E050E00E94A12600E00B
:1042500010E0EA18FB080C091D09A80197010E944B
:104260000927C901DA019C01AD0120573E4F4F4F8C
:104270005F4F5CC083E00E941E153E01882477FCDE
:104280008094982C8C179D0748F182E00E941E159F
:104290005C01CC24DD2483E00E941E157C016A1899
:1042A0007B088C089D08C401B30128EC30E040E095
:1042B00050E00E94A12600E010E0EA18FB080C097B
:1042C0001D09A80197010E940927C901DA019C0173
:1042D000AD01285A3D4F4F4F5F4F28C083E00E94E9
:1042E0001E155C01CC24DD2484E00E941E157C0197
:1042F0006A187B088C089D08C401B30128E730E0E8
:1043000040E050E00E94A12600E010E0EA18FB081F
:104310000C091D09A80197010E940927C901DA01AA
:104320009C01AD01205E3C4F4F4F5F4F999B02C0F7
:104330002FEF3FEFA898A89AA898A89AA898AE9AA5
:10434000C901DF91CF911F910F91FF90EF90DF9006
:10435000CF90BF90AF909F908F907F906F90089577
:10436000BC01009751F01092A8018EE790E20E94E4
:10437000F40D8091A8018823E1F30E94872020E0BA
:104380008F5F9F4F09F421E02093A701822F0895AA
:10439000FC017183608353834283178216821582E6
:1043A00014820895CF93DF93EC018C819D81892B3A
:1043B00011F4E0E018C08E819F81E881F981E80F57
:1043C000F91FE08101969F838E836A817B81861726
:1043D000970720F00E94C0269F838E838C819D8149
:1043E00001979D838C838E2FDF91CF910895FC01DF
:1043F0009B018481958168177907B0F48681978144
:10440000860F971F9783868362817381861797072C
:1044100020F00E94C0269783868384819581821B29
:10442000930B958384830895158214820895FC016B
:10443000CB012681378162817381820F931F0E9495
:10444000C0260190F081E02DE80FF91F80810895CA
:10445000CF93DF93EC01462F2C813D813093AA014D
:104460002093A9016A817B812617370710F080E02D
:1044700011C08E819F81820F931F0E94C026E88108
:10448000F981E80FF91F40838C819D8101969D83FE
:104490008C838FEFDF91CF9108950F931F93CF936C
:1044A000DF938C01EB0104C0C8010E9428222196F1
:1044B00068816623C9F78FEFDF91CF911F910F912C
:1044C0000895FC0140E02481358182819381281781
:1044D000390708F441E0842F0895FC0140E084810D
:1044E0009581860F971F228133818217930708F4E5
:1044F00041E0842F0895FC0184810895FC01158218
:10450000148208958091AF0108958091AF01809346
:10451000AE01089580E00E94ED241092AE0108954E
:10452000882329F08091AF018093AE0108950E9405
:104530008A220895853608F084E68093AE01809340
:10454000AF01882311F40E94ED2408958091AE01FB
:104550008823A9F08091AD018F5F8093AD018536EE
:1045600028F081E08093AD010E94ED249091AD018F
:104570008091AE01891718F480E00E94ED2408951F
:104580001092AD011092AE011092AF019AE0899F96
:10459000B001112486EA92E20E942F0E9093AC01A2
:1045A0008093AB0108959093B1018093B001089579
:1045B000E091B001F091B10109950895CF93DF9397
:1045C000EC01009739F409C02196E091B001F09117
:1045D000B101099588818823B9F7DF91CF910895BA
:1045E000CF93DF93EC01009731F40AC0E091B00162
:1045F000F091B1010995FE01219684918823B1F7CC
:10460000DF91CF910895E091B001F091B1018DE07B
:104610000995E091B001F091B1018AE00995089502
:104620000E94F0220E94032308952F923F924F92FE
:104630005F926F927F928F929F92AF92BF92CF9232
:10464000DF92EF92FF920F931F93DF93CF93CDB73B
:10465000DEB7A3970FB6F894DEBF0FBECDBF6AA337
:10466000242E2BA337014801442351F017FF08C023
:10467000EE24FF248701E618F7080809190902C08B
:10468000840173012AA1215090E0211091E0291B9F
:1046900029A318A2A82EBB24CC24DD24C801B7016D
:1046A000A60195010E94E726FB01E25FFB4F6491A2
:1046B0006F8FC801B701A60195010E94E726C901C5
:1046C000DA017C018D018EE1482E512C4C0E5D1ECD
:1046D00039A023C0E114F10401051105B9F0C801A6
:1046E000B701A60195010E94E726FB01E25FFB4F9F
:1046F0006491D2016C93C801B701A60195010E9493
:10470000E726C901DA017C018D0103C02BA1F2016A
:1047100020833A940894410851083320D9F6CE01F9
:104720004F968C01A9A10A1B1109222019F197FEAD
:1047300005C08DE2F80182938F011CC0C80101976A
:10474000611471048104910429F08C018BE2D80179
:104750008C9310C08C0180E2F80180830BC0E09143
:10476000B001F091B101D8018D918D010995BAA1E7
:10477000B150BAA3EAA1EE2391F7A3960FB6F8942D
:10478000DEBF0FBECDBFCF91DF911F910F91FF9084
:10479000EF90DF90CF90BF90AF909F908F907F90E1
:1047A0006F905F904F903F902F90089590930302E9
:1047B0008093020208959B01AC016050704F814FBD
:1047C0009F4FF3E0660F771F881F991FFA95D1F767
:1047D000E4E0220F331F441F551FEA95D1F70E94D2
:1047E000E726215029B9089581E792E008958AE7E4
:1047F00092E00895982F809170028823E1F39CB98C
:10480000109270020895982F809170028823E1F32E
:104810009CB91092700281E090E0089510927602A7
:1048200010927502089520E08091750290917602B1
:10483000892B09F421E0822F08951F920F920FB661
:104840000F9211242F933F934F935F936F937F9316
:104850008F939F93AF93BF93EF93FF936CB181E7D7
:1048600092E00E942822FF91EF91BF91AF919F911A
:104870008F917F916F915F914F913F912F910F9009
:104880000FBE0F901F901895682F8AE792E00E9444
:10489000282208951F920F920FB60F9211242F9382
:1048A0003F934F935F936F937F938F939F93AF93B8
:1048B000BF93EF93FF9380917902882371F08091E9
:1048C0007E0290917F02892B31F08AE792E00E946C
:1048D000D2218CB905C01092790281E080937002D8
:1048E000FF91EF91BF91AF919F918F917F916F91C8
:1048F0005F914F913F912F910F900FBE0F901F909E
:10490000189580917E0290917F02892B99F0809179
:104910007902882379F481E0809379028AE792E032
:104920000E94D221982F809170028823E1F39CB9D4
:10493000109270020895CF93DF93EC01809173027F
:1049400090917402892B69F08091750290917602A2
:10495000892B39F081E792E00E94D221888381E09F
:1049600001C080E0DF91CF91089581E792E062EB92
:1049700071E048E250E00E94C8218AE792E06AEDC7
:1049800071E048E250E00E94C8210895EF92FF9242
:104990000F931F937B018C010E94B5241092030298
:1049A0001092020288ED8AB960E875E280E090E03A
:1049B0000E94DB2381E080937002109279021092B2
:1049C0008302109282027894C801B7010E94DB230F
:1049D0001F910F91FF90EF900895882319F0AF9ADF
:1049E000C5980895AF98C59A089580E0089520E08D
:1049F00080910702882309F421E020930702909117
:104A00000502992351F0222321F088B3892B88BB1A
:104A1000089588B39095982398BB0895C79A0895F0
:104A2000809104020895282F80930402909105023A
:104A3000907E9093050230910602307E30930602FC
:104A400088B38F6188BB253079F1263070F422302D
:104A5000C1F0233020F4213009F054C010C02330BD
:104A600091F0243009F04EC016C02730B1F1273044
:104A700000F12830E9F1293009F044C006C0906106
:104A800005C0926003C0946001C0986090930502D5
:104A90003093060208950E945213909105022091CE
:104AA0000602882371F013C090930502832F826061
:104AB00018C00E945213909105022091060288238B
:104AC00031F09E7F90930502822F81600AC09B7F08
:104AD00090930502822F846004C090930502832F77
:104AE00088608093060298B38095892388BB0895D7
:104AF00090930502832F80618093060298B380957E
:104B0000892388BB0895BC01C7988EE095E20E9476
:104B1000F40D089510920C02809105028E7F80930F
:104B200005028091060281608093060298B3809509
:104B3000892388BB86EC95E268EE73E00E942F0E15
:104B400090930B0280930A0280910C028630E0F36E
:104B50000895A79AAF9887B38F6B87BB80910502A2
:104B6000807480930502809106028074809306020F
:104B700088B38F6B88BB87EF94E264EF71E00E948B
:104B80002F0E9093090280930802089580910C02E1
:104B90008F5F80930C0280910C02833031F184305E
:104BA00030F4813061F0823009F05BC013C0853091
:104BB00091F1853028F1863009F053C03DC08091D5
:104BC00006028E7FC09A909105029C7F9093050209
:104BD00082602BC0809106028D7FC19A9091050260
:104BE000997F90930502846020C0809106028B7F9C
:104BF000C29A90910502937F90930502886015C038
:104C000080910602877FC39A90910502977E9093C8
:104C1000050280610AC0809106028F7EC49A90913D
:104C200005029F7C9093050280628093060298B3F0
:104C30008095892388BB0895809105028F7D80939C
:104C40000502809106028F7D80930602C59A88EE48
:104C500093E00E94832580910A0290910B020E94AA
:104C60006B0E0895FC0188279927E8942191203242
:104C7000E9F3293010F02E30C8F32B3241F02D32F9
:104C800039F4689404C00E949926820F911D2191E5
:104C900020532A30C0F31EF4909581959F4F0895BC
:104CA000FB01DC0102C005900D9241505040D8F745
:104CB0000895FB01DC0105900D920020E1F70895B5
:104CC000FB01DC014150504030F08D910190801982
:104CD00019F40020B9F7881B990B0895DF92EF9221
:104CE000FF920F931F937B018C01FB010995D82E36
:104CF000C8010196F7010995982F8D2D1F910F91ED
:104D0000FF90EF90DF900895DF92EF92FF920F9364
:104D10001F93D72E7A018C01FA010995C8010196DB
:104D20006D2DF70109951F910F91FF90EF90DF9086
:104D300008957AE0979F902D879F802D910D1124E3
:104D40000895629FD001739FF001829FE00DF11DD5
:104D5000649FE00DF11D929FF00D839FF00D749FF5
:104D6000F00D659FF00D9927729FB00DE11DF91FA1
:104D7000639FB00DE11DF91FBD01CF0111240895FE
:104D8000AA1BBB1B51E107C0AA1FBB1FA617B70771
:104D900010F0A61BB70B881F991F5A95A9F780958D
:104DA0009095BC01CD01089597FB092E07260AD0E6
:104DB00077FD04D0E5DF06D000201AF470956195E8
:104DC0007F4F0895F6F7909581959F4F0895A1E242
:104DD0001A2EAA1BBB1BFD010DC0AA1FBB1FEE1F75
:104DE000FF1FA217B307E407F50720F0A21BB30BC0
:104DF000E40BF50B661F771F881F991F1A9469F73C
:104E000060957095809590959B01AC01BD01CF0197
:104E1000089597FB092E05260ED057FD04D0D7DF45
:104E20000AD0001C38F450954095309521953F4F9D
:104E30004F4F5F4F0895F6F7909580957095619567
:0C4E40007F4F8F4F9F4F0895F894FFCFD5
:104E4C00A704F800FF001D0124014201490167017C
:104E5C006E018C019301B101B801D601DD01FB019A
:104E6C0002022002270245024C026A0271028F02E2
:0A4E7C009602B402BB020000000021
:00000001FF
